:020000040000FA
:040000006A303A2800
:08000800A000030EA100831209
:1000100005191028831601178312B23081002B288E
:1000200083160113831203140B190310A80DA90DD5
:10003000AA0DAB0DAC0DAC16FF302C02031D2B2806
:10004000FA302B02031D2B2831152A08AF0029088E
:10005000AE002808AD008B100B11210E8300A00EFE
:04006000200E090065
:0C007400203084008001840A6030040207
:10008000031C3C281230B0005E2283160C3085051C
:1000900087018312850187010730990000309A009B
:1000A000103083168E008312603083168F00831207
:1000B0000030831691008312C830831681008312AA
:1000C00031309000003083168C00831210308B008A
:1000D000831600309B001C141A088312BC00851D77
:1000E0006B233C1C8228831610309B001C141A08BA
:1000F0008312BD00831630309B001C141A08831233
:10010000C200F522831620309B001C141A088312AB
:10011000C1000130C1080319C10081018E018F01A6
:100120000B118B100B108C018B17A5203119A820F7
:100130003B22B30BA328031085190314B90DF0302B
:1001400039020319CA210A239528640032100800D5
:1001500031110130B7008B132030370783169B0015
:100160001C141A088312A4001030370783169B0052
:100170001C141A088312A300A6000230A606003041
:10018000370783169B001C141A088312A200A700CD
:100190000130A7068B17321CD32822090339A2008D
:1001A000A309A409A50924082F02031DC4292308B3
:1001B0002E02031D4D2922082D02031DC4290130E2
:1001C0003702031DEA283C19E9283D18EA283D14A6
:1001D0003E145F2202303702031DF5283C19F42833
:1001E000BD18F528BD143E14662203303702031DE6
:1001F00000293C19FF283D1900293D153E146D22A8
:1002000004303702031D0B293C190A29BD190B299B
:10021000BD153E14742205303702031D16293C1902
:1002200015293D1A16293D163E147B220630370249
:10023000031D21293C192029BD1A2129BD163E1470
:10024000822207303702031D2C293C192B293D1B24
:100250002C293D173E14892208303702031D372907
:100260003C193629BD1B3729BD173E149022093091
:100270003702031D42293C194129421842294214E0
:100280003E1497220A303702031D4D293C194C2990
:10029000C2184D29C2143E149E2226082E02031DA8
:1002A000C42927082D02031DC42901303702031D6C
:1002B00060293C195F293D1C60293D103E14A52290
:1002C00002303702031D6B293C196A29BD1C6B29BA
:1002D000BD103E14A92203303702031D76293C19B4
:1002E00075293D1D76293D113E14AD22043037029B
:1002F000031D81293C198029BD1D8129BD113E1492
:10030000B12205303702031D8C293C198B293D1E73
:100310008C293D123E14B52206303702031D972961
:100320003C199629BD1E9729BD123E14B9220730EB
:100330003702031DA2293C19A1293D1FA2293D1303
:100340003E14BD2208303702031DAD293C19AC29EB
:10035000BD1FAD29BD133E14C12209303702031D54
:10036000B8293C19B729421CB82942103E14C522AD
:100370000A303702031DC3293C19C229C21CC329F4
:10038000C2103E14C922C429B70A0B303702031821
:100390000800AB280130B600B300B400B500B700C8
:1003A00085018701B113A520B30B0A2A0310851913
:1003B0000314B90DF03039020319312AB40B0A2A9B
:1003C000013037020319CD22023037020319D1223E
:1003D000033037020319D522043037020319D9221A
:1003E000053037020319DD22063037020319E122F6
:1003F000073037020319E522083037020319E922D2
:10040000093037020319ED220A3037020319F122AD
:100410009630B400311DD3293111321C142A2D0914
:100420000339AD00AE09AF092F1CD3298E018F010E
:100430000C1CD3290C102E1ED3298B132030370708
:10044000BB002F08BA00492210303707BB002E0826
:10045000BA00492200303707BB002D08BA004922F4
:100460008B1785018701B70AB6010B303702031CD1
:10047000D329F52208003E1C08003E101030BB00B6
:100480003D08BA0049223030BB004208BA00492278
:1004900008008B133A0883161C159A0083123B0838
:1004A00083169B0055309D00AA309D009C1464006B
:1004B0009C18572A1C1183128B1708000800051678
:1004C00040084107D0000F08D100080085164008F9
:1004D0004107D2000F08D300080005144008410767
:1004E000D4000F08D5000800851440084107D60045
:1004F0000F08D7000800871440084107D8000F08EC
:10050000D9000800071540084107DA000F08DB0092
:100510000800071440084107DC000F08DD00080050
:10052000871640084107DE000F08DF0008000716A5
:1005300040084107CC000F08CD000800871540088F
:100540004107CE000F08CF00080005128E018F0171
:10055000080085128E018F01080005108E018F01A1
:10056000080085108E018F01080087108E018F0111
:10057000080007118E018F01080007108E018F01FE
:10058000080087128E018F01080007128E018F016B
:10059000080087118E018F0108000508103A8500B8
:1005A00008000508203A850008000508013A850082
:1005B00008000508023A850008000708023A87008B
:1005C00008000708043A870008000708013A870076
:1005D00008000708203A870008000708103A87003B
:1005E00008000708083A870008003D180516BD18DE
:1005F00085163D190514BD1985143D1A8714BD1AB9
:1006000007153D1B0714BD1B871642180716C21895
:10061000871508003C1D080050084002031D152BDB
:1006200051080F02031C152B051252084002031D2E
:100630001E2B53080F02031C1E2B85125408400268
:10064000031D272B55080F02031C272B05105608E6
:100650004002031D302B57080F02031C302B85105E
:1006600058084002031D392B59080F02031C392B6F
:1006700087105A084002031D422B5B080F02031C1F
:10068000422B07115C084002031D4B2B5D080F0233
:10069000031C4B2B07105E084002031D542B5F0800
:1006A0000F02031C542B87124C084002031D5D2BC4
:1006B0004D080F02031C5D2B07124E084002031D5C
:1006C000662B4F080F02031C662B87110C1C0800B9
:1006D0000C10C00A0800B601B301B4013C1C732B16
:1006E000BC01BC147A2BBC1C782BBC013C157A2BAA
:1006F000BC013C143C08B60064007E2B7F2B802B91
:10070000812B822BB41B0516B41F0512B30B7C2B57
:10071000B40B7C2B0310B60CB608031D7C2B0030E9
:0A072000BB003C08BA0049220800A3
:084000000900030002000600A4
:02400E00CC33B1
:10420000010078007A007C007E007B0079007F004E
:104210007D007A0078007E007C00FF00FF00FF0038
:104220000000F200F600FA00FE00F200F600FA00CC
:10423000FE00F200F600FA00FE00FF00FF00FF00A3
:10424000010005000500050005000900090009003E
:1042500009000D000D000D000D00FF00FF00FF0024
:10426000FF00FF00FF00FF00FF00FF00FF00FF0056
:10427000FF00FF00FF00FF00FF00FF00FF00FF0046
:10428000FF00FF00FF00FF00FF00FF00FF00FF0036
:10429000FF00FF00FF00FF00FF00FF00FF00FF0026
:1042A000FF00FF00FF00FF00FF00FF00FF00FF0016
:1042B000FF00FF00FF00FF00FF00FF00FF00FF0006
:1042C000FF00FF00FF00FF00FF00FF00FF00FF00F6
:1042D000FF00FF00FF00FF00FF00FF00FF00FF00E6
:1042E000FF00FF00FF00FF00FF00FF00FF00FF00D6
:1042F000FF00FF00FF00FF00FF00FF00FF00DD00E8
:00000001FF
